S10C0100160246000000E000FFB5
S123034910CE03498E0109108E0000C60010AF815A26FACC0006FDE11ECC0002FDE11EBD5B
S12303690487CC00E0FDE10CBD04878E0648BD062B8E0672BD062BBD062F81522764814E2A
S1230389273D815027488157102700A5814D272A815127228172274A816E27238170272EDB
S12303A981771027008B816D2710817127088E073BBD062320BB6E9FF800BD052A20B2BE1E
S12303C901043001BF0104262A7C01032025BE010426087D0103271B7A0103301FBF0104BC
S12303E920118E06E9BD0623BD05902941F70103BF01044FC601FDE104F60105FDE106F613
S12304090104FDE108F60103FDE10AC620FDE10EBD04878E0109108E0100BD0496FCE1007D
S1230429E780A780313F26F2BD0487BD049E7E037A8E06E9BD0623BD0590293FF70103BF20
S123044901044FC601FDE104F60105FDE106F60104FDE108F60103FDE10ACC0030FDE10E07
S1230469BD04878E0109108E0100BD0496E680A680FDE100313F26F2BD04877E037AFCE187
S12304890EC58026F9FCE10EC54027F239FCE10EC50827F9398E0702BD0623B60103BD0591
S12304A9F8BE0104BD05F0BD0627108E000030A900FFBD04CF8E0744BD0623BD0638108E7A
S12304C9010030A900FF1F10C30010C4F034061F20C4F01F01ACE42705170157270332624A
S12304E93934108E072F170131AEE41700F9170146C610A689010930011700F317013A5A6F
S123050926F1170132AEE1C610A6890109300181202504817E2302862E17011F5A26EA203B
S1230529B48E0714BD062317007429348C0200242F1F128E072F1700E11F211700A917009E
S1230549F8A6A901091700A71700EE1700602811810827DF811827DB815E2721810D2613B2
S123056939A7A90109A1A9010927081700CB863F1700C8108C01FF27BA312120B6108C0091
S12305890027B0313F20AC327D8D232957A7E48D1D2951A7618D17294BA7624F35948D21BE
S12305A929421F018D08293C3410A76135908D112932484848481F898D0729283404ABE02F
S12305C9398D638130251D813922038030398141251281462203803739816125078166223E
S12305E9038057391A0239341035028D0235023402444444448D043502840F8B3081392F00
S1230609028B0720363402C608A68068E42502862D8D288D245A26F135826E9FF8106E9FE3
S1230629F80E6E9FF80C7D010827046E9FF8066E9FF8046E9FF8088D0086206E9FF80A0A78
S12306490D434F4D5041435420464C41534820534543544F5220524541442F575249544505
S1230669205554494C495459040D0A285229205245414420534543544F5220202028572927
S123068920575249544520534543544F5220200D0A284E29204E45585420534543544F526D
S12306A9202020285029205052455620534543544F522020200D0A284D29204D4F4449463B
S12306C95920534543544F52202851292051554954202020202020202020200D0A3A2004EA
S12306E9534543544F52204E554D4245522028362048455829203A2004534543544F52201A
S12307094E554D424552202D2024040D0A4D454D4F52592041444452455353202833204875
S12307294558293A2004202D200400000A0D0000000457686174203F0D0A040D0A486974B2
S118074920616E79206B657920746F20636F6E74696E7565043A
S9030000FC
